:100000000C942D090C944A090C944A090C944A0941
:100010000C944A090C944A090C944A090C944A0914
:100020000C944A090C944A090C946C2B0C943E2CA9
:100030000C9494250C944A090C944A090C944A098E
:100040000C944A090C944A090C944A090C944A09E4
:100050000C944A090C941C260C944A090C944A09E5
:100060000C944A090C944A090C944A090C944A09C4
:100070000C944A090C944A090C944A090C944A09B4
:100080000C944A090C944A090C944A090C944A09A4
:100090000C944A090C944A090C944A090C944A0994
:1000A0000C944A090C944A090C944A09DB0DDB0DA7
:1000B000070E070E6F0E8D0EA50FA50F980E310FB0
:1000C000420F420FAB2CD22CCA2DD22CCA2D1E2D82
:1000D000412DCA2D982DA72D29001E001F0020009C
:1000E00021002200230024002500260027002D00E7
:1000F0002E002B0014001A000800150017001C0029
:1001000018000C00120013002F003000350004000E
:100110001600070009000A000B000D000E000F007A
:10012000330034003100E1001D001B0006001900FF
:100130000500050010003600370038002800520086
:10014000000FE000E200E300AA5D2C000000AB5DC0
:100150002A00E50050004F00510035001E001F002E
:100160002000210022002300240025002600270073
:100170002A0001002B0014001A00090013000A00D5
:100180000D000F0018001C0033004C000100290076
:10019000040015001600170007000B0011000800EE
:1001A0000C00120034000100E1001D001B000600DD
:1001B000190005000500100036003700380028003F
:1001C0000100AC5DE000E200E300AA5D2C0000004D
:1001D000AB5D5000510052004F00010035001E0081
:1001E0001F002000210022002300240025002600FB
:1001F00027002A0001002B003400360037001300CE
:100200001C0009000A00060015000F004C00010048
:10021000290004001200080018000C0007000B0061
:1002200017001100160038000100E100330014002F
:100230000D000E001B001B0010001A0019001D000D
:1002400028000100AC5DE000E200E300AA5D2C00A4
:100250000000AB5D5000510052004F00010035021C
:100260001E021F0220022102220223022402250272
:10027000260227022A00010035021E021F02200268
:1002800021022202230224022502260227024C0018
:1002900001004C003A003B003C003D003E003F00A6
:1002A0002D022E022F023002310201000100400017
:1002B0004100420043004400440032026402010055
:1002C0000100010001000100010001000100010026
:1002D000010000000100AB00AA00A900AE0001006F
:1002E00035001E001F0020002100220023002400F2
:1002F0002500260027002A00010035001E001F00EF
:1003000020002100220023002400250026002700D1
:100310004C0001004C003A003B003C003D003E0018
:100320003F002D002E002F003000310001000100A1
:100330004000410042004300440044003200640099
:1003400001000100010001000100010001000100A5
:100350000100010000000100AB00AA00A900AE00EE
:10036000010000000000000000000000000000008C
:10037000000000000000000000000000000000007D
:10038000000000000000000000000000000000006D
:10039000000000000000000000000000000000005D
:1003A000000000000000000000000000000000004D
:1008F00000000000000000003A003B003C003D000A
:100900003E003F00400041004200430044004500DB
:1009100001000100005C0100010001000100010074
:1009200001000100010001004C0001000100010074
:1009300001001D5C1E5C135C0A5CA75DA85DA95DDF
:1009400001000100010001002B5C2A5C265C275C91
:100950002C5C2C5C01000100010001000100010081
:100960000100010001000100010001000000010080
:100970000100010001000100010044454255473AD1
:100980002064697361626C65642E0A0044454255B7
:10099000473A20656E61626C65642E0A000A002584
:1009A000303258006C65645F7461736B3A20004F9D
:1009B0006E6573686F743A206163746976653A2076
:1009C00025640A000A002530313662003A200025ED
:1009D000303258000A722F632030313233343536CA
:1009E0003738394142434445460A00290A002575F3
:1009F000002F002575005D28002564002000256477
:100A000000200025640020002564007C0025303291
:100A100058006D6F7573656B6579205B62746E7CD1
:100A2000782079207620685D287265702F61636C6C
:100A3000293A205B00313A0964656C6179282A31D2
:100A4000306D73293A2025750A323A09696E74654A
:100A50007276616C286D73293A2025750A333A093C
:100A60006D61785F73706565643A2025750A343A64
:100A70000974696D655F746F5F6D61783A202575E3
:100A80000A353A09776865656C5F6D61785F7370E8
:100A90006565643A2025750A363A09776865656C9C
:100AA0005F74696D655F746F5F6D61783A2025755D
:100AB0000A00703A097072696E742076616C75650F
:100AC000730A643A097365742064656661756C74B1
:100AD000730A75703A092B310A646E3A092D310A8E
:100AE0006C743A092B31300A72743A092D31300A8C
:100AF0004553432F713A09717569740A0A73706519
:100B00006564203D2064656C7461202A206D6178E5
:100B10005F7370656564202A202872657065617452
:100B2000202F2074696D655F746F5F6D6178290A8D
:100B300077686572652064656C74613A20637572CC
:100B4000736F723D25642C20776865656C3D256464
:100B50000A53656520687474703A2F2F656E2E777E
:100B6000696B6970656469612E6F72672F77696B55
:100B7000692F4D6F7573655F6B6579730A004D3E24
:100B800020004D25753A25733E20003F0A003D2088
:100B900025750A003F0A0064656661756C74730A06
:100BA0000025750A003F0A000A092D2056616C7560
:100BB0006573202D0A00710A000A092D204D6F75FA
:100BC00073656B6579202D0A003F00433E20004C81
:100BD00025640A000A092D20537461747573202D51
:100BE0000A686F73745F6B6579626F6172645F6CC2
:100BF00065647328293A20253032580A6B6579627A
:100C00006F6172645F70726F746F636F6C3A2025EE
:100C10003032580A6B6579626F6172645F69646C27
:100C2000653A20253032580A74696D65725F7265C5
:100C30006164333228293A202530386C580A000A7A
:100C4000092D2056657273696F6E202D0A5649442E
:100C50003A203078424238302848657877697265A2
:100C600029205049443A20307830353044284F729A
:100C700074686F203578313329205645523A203038
:100C800078303030310A4255494C443A20202846C9
:100C900065622032372032303232290A4F505449AF
:100CA0004F4E533A204C554641204D4F5553454BDE
:100CB00045592045585452414B455920434F4E53B6
:100CC0004F4C4520434F4D4D414E44203531320A63
:100CD0004743433A20352E342E30204156522D4C76
:100CE0004942433A20322E302E30204156525F4145
:100CF0005243483A20617672350A000A092D204392
:100D00006F6E736F6C65202D0A4553432F713A093E
:100D1000717569740A6D3A096D6F7573656B6579E4
:100D20000A000A092D204D61676963202D0A443AA3
:100D3000094465627567204D65737361676520546A
:100D40006F67676C650A583A094D6174726978205B
:100D50004465627567204D6F646520546F67676CEA
:100D600065202D2053686F77206B657970726573ED
:100D700073657320696E206D617472697820677283
:100D800069640A4B3A094B6579626F617264204469
:100D90006562756720546F67676C65202D20536806
:100DA0006F77206B65797072657373207265706FF1
:100DB00072740A4D3A094465627567204D6F757308
:100DC0006520546F67676C650A563A0956657273F9
:100DD000696F6E0A533A095374617475730A433A22
:100DE00009416374697661746520436F6E736F6C3B
:100DF00065204D6F64650A46312D4631303A0953FE
:100E0000776974636820746F204C61796572203053
:100E10002D392028463130203D204C30290A302DF4
:100E2000393A0953776974636820746F204C61798B
:100E3000657220302D390A47524156453A09537799
:100E40006974636820746F204C617965722030206A
:100E500028616C7465726E617465290A423A094AA8
:100E6000756D7020746F20426F6F746C6F61646574
:100E7000720A4553433A094A756D7020746F2042D7
:100E80006F6F746C6F616465722028616C74657239
:100E90006E617465290A453A095072696E7420457D
:100EA0004550524F4D2053657474696E67730A4202
:100EB00053504143453A09436C65617220454550A2
:100EC000524F4D0A006B65796D61705F636F6E669E
:100ED00069672E7261773A20253032580A2E73776F
:100EE00061705F636F6E74726F6C5F636170736C5F
:100EF0006F636B3A2025750A2E636170736C6F63A4
:100F00006B5F746F5F636F6E74726F6C3A202575E0
:100F10000A2E737761705F6C63746C5F6C677569C0
:100F20003A2025750A2E737761705F7263746C5F67
:100F3000726775693A2025750A2E737761705F6C48
:100F4000616C745F6C6775693A2025750A2E73773A
:100F500061705F72616C745F726775693A202575A4
:100F60000A2E6E6F5F6775693A2025750A2E7377B2
:100F700061705F67726176655F6573633A2025759E
:100F80000A2E737761705F6261636B736C61736863
:100F90005F6261636B73706163653A2025750A2E29
:100FA0006E6B726F3A2025750A0064656275675F23
:100FB000636F6E6669672E7261773A20253032580A
:100FC0000A2E656E61626C653A2025750A2E6D6188
:100FD000747269783A2025750A2E6B6579626F61A3
:100FE00072643A2025750A2E6D6F7573653A202557
:100FF000750A006565636F6E6669673A0A646566BF
:1010000061756C745F6C617965723A2025750A00B0
:101010003F000A6D6F7573653A206F66660A000AB5
:101020006D6F7573653A206F6E0A000A6B657962A1
:101030006F6172643A206F66660A000A6B657962B6
:101040006F6172643A206F6E0A000A6D6174726992
:10105000783A206F66660A000A6D61747269783AA0
:10106000206F6E0A000A64656275673A206F6666D3
:101070000A000A64656275673A206F6E0A000A0A00
:101080004A756D70696E6720746F20626F6F746C43
:101090006F616465722E2E2E2000433E2000436C4B
:1010A000656172696E6720454550524F4D0A000ACE
:1010B000002530325820006B6579626F6172645F81
:1010C0007265706F72743A20005B735D005B575DF0
:1010D000005B535D005B525D005B445D005B435D04
:1010E0000016034F007200740068006F0020003586
:1010F00000780031003300000010034800650078DC
:10110000007700690072006500000004030904090B
:10111000025B00030100A0FA0904000001030101C1
:101120000009211101000122400007058103080088
:10113000010904010001030000000921110100015F
:10114000227B00070582032000010904020002033C
:10115000000000092111010001222200070583037C
:101160002000010705030320000112010002000016
:10117000000880BB0D050100010200010631FF09D6
:1011800074A1010975150026FF00952075088102DC
:101190000976150026FF00952075089102C005010B
:1011A0000902A10185020901A10005091901290807
:1011B00015002501950875018102050109300931E5
:1011C0001581257F95027508810609381581257FCF
:1011D000950175088106050C0A38021581257F9551
:1011E0000175088106C0C005010980A101850319A8
:1011F000012AB700150126B700950175108100C0BE
:10120000050C0901A101850419012AA00215012676
:10121000A002950175108100C005010906A1010514
:101220000719E029E7150025019508750181029548
:1012300001750881010507190029FF150026FF0027
:1012400095067508810005081901290595057501A0
:101250009102950175039101C00011241FBECFEFCB
:10126000DAE0DEBFCDBF11E0A0E0B1E0E0E1FDE5F6
:1012700002C005900D92AA3FB107D9F722E0AAEF6C
:10128000B1E001C01D92AB3EB207E1F70E94EB1B3B
:101290000C94862E0C940000FF93EF93E091FA01DA
:1012A000F091FB01309709F00995EF91FF910895B6
:1012B000FC018591803011F0EFDFFBCF0895FF270F
:1012C000E0E230E247FF0CC0419597FF09C0EDE234
:1012D0006095709580959095611D711D811D911D82
:1012E00027FF02C0219530E350E2AA27660F771F3F
:1012F000881F991FAA1FA41710F0A41B63955A9565
:10130000A9F7AA3008F0A95FA05DAF93F395611526
:1013100071058105910541F7ED3211F4EF93F395D5
:10132000F21718F43F93F395FBCF8F91B5DFFA9541
:10133000E1F70895E991F9918591803021F08532A6
:1013400019F0AADFF9CF089520E0E89455915532BD
:10135000C1F3503311F4689455915A3348F4505303
:1013600090F3220F022E220F220F200D250FF4CF13
:101370000EF4219589919991533619F3533729F138
:10138000533559F1BC0188279927E8945C3621F43C
:101390008991999168945591543639F446EF7EF0CD
:1013A00077FF0DC08FEF9FEF0AC055374AE039F045
:1013B000583540E121F0523642E009F00895FF939C
:1013C000EF937DDFEF91FF91B7CFFF93EF93FC0198
:1013D00081918030B9F360DFFBCFFF93EF9368DF3B
:1013E000F1CFDF93CF93CDB7DEB72596A3DFCF91B3
:1013F000DF910895CF93DF93EC010E949216BE0116
:1014000080E090E0DF91CF910C948D10CF93FB01A1
:10141000893A2DE5920701F140F4873A2DE59207CC
:1014200069F0883A9D4581F03FC08B3A2DE59207DF
:10143000E1F0C0F08C3A9D4561F136C0C281CC2309
:10144000A1F181E090E005C0C281CC2371F182E07E
:1014500090E00E94FA0923C0C281CC2331F184E0DC
:1014600090E0F7CFC28183E002C0C28184E0CC2348
:1014700041F00E94ED1040E164E083E00E94FD0A2B
:101480000EC00E940E1140E164E083E00E94FD0A5C
:101490000CC0C28185EECC2321F00E945B0CC0E021
:1014A00004C00E940A0D01C0C1E08C2FCF910895A5
:1014B000089581E008950C94060A08950C945D0A3D
:1014C0001F93CF93DF9300D000D01F92CDB7DEB72C
:1014D00049835A836B833091FD0189819A8131114F
:1014E00014C0662359F0222349F00E94E211182FFC
:1014F000682F89819A810E948B1103C00E94B611C6
:10150000182F69817A81812F04C00E94E2116981BC
:101510007A810F900F900F900F900F90DF91CF91E5
:101520001F910C942B19FC01262F4081518162815F
:10153000738184810C94600A81E00895CF93DF93D6
:10154000EC0160E00E94930ABE01DF91CF910C9400
:101550005E0A8F929F92AF92BF92CF92DF92EF92EC
:10156000FF920F931F936B017C0181E090E0A0E05C
:10157000B0E04C015D0104C0880C991CAA1CBB1C86
:101580004A95D2F7AC01BD0104C0440F551F661F38
:10159000771F2A95D2F7482959296A297B2904C03F
:1015A000880F991FAA1FBB1F0A95D2F78A019B01BA
:1015B0000C211D212E213F2140175107620773077F
:1015C00039F4BC01CD016C297D298E299F290AC0DF
:1015D00080959095A095B095BC01CD016C217D21A1
:1015E0008E219F211F910F91FF90EF90DF90CF9060
:1015F000BF90AF909F908F9008950F93382F262F14
:1016000060912B0270912C0280912D0290912E02FC
:10161000042F432F0E94A90A0F910C94C7100C9419
:101620009C1A0C949A1A08950E9435100E94130B6C
:101630002FEF84E39CE0215080409040E1F700C010
:1016400000000C9442260F931F93CF93DF938C01DD
:1016500061E00E94930AEC01B8010E945B0A8823B2
:1016600009F45BC0B801CE010E942124882309F44B
:1016700054C0B801CE010E94031F882309F44DC055
:10168000B801CE010E947D23882309F446C0F801E9
:1016900082818823D9F1CF3D8CE5D80779F140F4D8
:1016A000C115FCE5DF0791F0C130DC4591F02EC09B
:1016B000CC35EDE5DE0741F1CD35FDE5DF0709F17C
:1016C000CB35DD4519F50E94791620C00E94140B18
:1016D00024C080919102C82FC095C170C0FB80F9D1
:1016E00080939102CC2329F08CE899E00E9458095C
:1016F00014C08AE799E00E94580910C00E942C1774
:101700000CC00E94701602C00E947C16C801DF91B6
:10171000CF911F910F910C94590AC0E08C2FDF914B
:10172000CF911F910F9108950E9476250C94D20BB2
:101730000E94D50B0C947C258295982F937344E0DE
:10174000949F900111248C7C86958695282B822F5E
:101750008575880F2A7A2695822B0895CF93DF937B
:10176000D92F0E949C0BC82F8D2F0E949C0B2C2FD1
:1017700030E0322F2227A901482BCA01DF91CF91F7
:10178000089508950C94C10B81E008950C94C40B46
:101790000895CF93C82F0E94C20B8C2F0E94C60BB6
:1017A000CF91089580E00C94C90B0E947D240C9485
:1017B000C90BCF930E947D24C82F8091FC01C817CC
:1017C00041F1C093FC018091910282FF1EC080FF15
:1017D00004C084EA99E00E9458098091910280FF38
:1017E0000CC01F92CF938FE999E09F938F930E9433
:1017F000F1090F900F900F900F908091910280FF50
:1018000004C08DE999E00E9458098C2FCF910C9467
:10181000C90BCF910895CF93DF93CDB7DEB72B9748
:101820000FB6F894DEBF0FBECDBF4F8358876987D0
:101830007A878B8761110E94A8159E012F5F3F4F09
:1018400086E0F90111928A95E9F785E0FE01379665
:10185000D90101900D928A95E1F789819A814C8195
:101860005D81452B31F09F3F31F491E08F3F19F4BA
:1018700003C091E001C090E090FF09C049815A8106
:101880006B817C818D819E810E94C91405C0C90134
:101890000E949C0A8111F2CF2B960FB6F894DEBFFE
:1018A0000FBECDBFDF91CF910895FC018081918162
:1018B0000E9424120895CF93882309F4A9C0C82F49
:1018C0008238C1F40E947D2481FDA2C069E3809129
:1018D0000201909103010E944E250E94CA152FEF2C
:1018E00081EE94E0215080409040E1F700C000007C
:1018F00069E319C0833801F50E947D2480FD88C00A
:1019000063E580910201909103010E944E250E949F
:10191000CA152FEF81EE94E0215080409040E1F70E
:1019200000C0000063E580910201909103010E94D4
:101930005025CF910C94CA158438C1F40E947D249F
:1019400082FD66C067E480910201909103010E94CC
:101950004E250E94CA152FEF81EE94E02150804061
:101960009040E1F700C0000067E4DDCF8CEF8C0F02
:10197000813AF8F48C2F0E942623811149C06C2FE4
:1019800080910201909103010E941825882349F05B
:101990006C2F80910201909103010E9450250E94BA
:1019A000CA156C2F80910201909103010E944E256F
:1019B000C0CF80E28C0F883048F4C77081E001C04E
:1019C000880FCA95EAF70E948B15B3CFEBE5EC0FB1
:1019D000E33040F4F0E0E95BFE4F808190E0CF918E
:1019E0000C94E024E8E5EC0FE73150F4F0E0EE0F62
:1019F000FF1FE75EFE4F80819181CF910C94F6240A
:101A0000CD3E30F08C2F0E94701CCF910C94421D63
:101A1000CF910895882309F464C0823879F40E9434
:101A20007D2481FF5EC069E38091020190910301F2
:101A30000E944E250E94CA1569E310C08338B1F494
:101A40000E947D2480FF4DC063E58091020190914A
:101A500003010E944E250E94CA1563E58091020190
:101A6000909103010E9450250C94CA15843879F492
:101A70000E947D2482FF35C067E48091020190912D
:101A800003010E944E250E94CA1567E4E7CF9CEF30
:101A9000980F913A10F4682FE1CF90E2980F9830A8
:101AA00050F4877091E001C0990F8A95EAF7892F69
:101AB0000E949115D9CF9BE5980F933020F480E0D8
:101AC00090E00C94E02498E5980F973120F480E0A2
:101AD00090E00C94F6248D3E20F00E94CB1C0C94D8
:101AE000421D08951F93CF93DF93182FEB010E949F
:101AF0005B0C209741F08FE99FE00197F1F700C060
:101B000000002197F6CF812FDF91CF911F910C9488
:101B10000A0D893319F060E070E002C060E570E002
:101B20000C94720D882321F00E948B150C94CA1519
:101B30000895882321F00E9491150C94CA150895E8
:101B4000CF92DF92EF92FF920F931F93CF93DF9389
:101B50007C01D62FC72FFC011281058102950F70E1
:101B60000E9481158823B9F01123A9F08C2F807F62
:101B7000803421F080E28D0F883068F08091C502BA
:101B800082FD09C082E00E942A160E94811591E020
:101B9000D82ED92601C0D12CCC2EC2948FE0C822D9
:101BA0008C2D90E08C30910508F0CFC1FC01EA5AF1
:101BB000FF4F0C941D2E8C2F807FCF70882311F047
:101BC000C295C07F112399F0CC2309F4AAC180E209
:101BD0008D0F883010F0D11104C08C2F0E948B150E
:101BE00003C08C2F0E949B150E94CA159AC18D2F8D
:101BF0000E940A0DCC2309F4A8C180E28D0F883021
:101C000038F1DD2329F18C2F0E94A11524C08C2FDF
:101C1000807FCF70803211F0C295C07FDD2319F034
:101C2000D130A1F13DC08091C50282FF17C01123C0
:101C300049F0CC2329F08C2F0E948B150E94CA15E5
:101C400080E070C180E00E940A0DCC2309F47DC1C0
:101C50008C2F0E9491150E94CA1577C1112371F033
:101C6000002341F0013031F40E94AB158C2B0E940F
:101C7000B3156BC10E94AB158C2B1DC0002319F04E
:101C8000013009F462C10E94C01525C0112321F062
:101C9000063008F05AC10EC0053008F056C11BC00E
:101CA000112361F0002331F0F701858180FF39C1F4
:101CB0008F7085838C2F0E94920D47C1002359F0AD
:101CC000D93309F03FC1FFEF07EE13E0F1500040B8
:101CD0001040E1F735C18C2F0E94990D36C18C2F31
:101CE00086958695837019F0813061F02EC111239D
:101CF00021F08D2F9C2F937002C080E090E00E9415
:101D0000E0242BC1112321F08D2F9C2F937002C052
:101D100080E090E00E94F62420C18D2F112319F05D
:101D20000E94701C02C00E94CB1C0E94421D15C163
:101D30008C2F837009F047C011110BC12D2F2295F4
:101D400026952770220F220F6D2F6F70862F90E03F
:101D5000A0E0B0E0022E04C0880F991FAA1FBB1F8D
:101D60000A94D2F7D4FF10C04FE050E060E070E07A
:101D700004C0440F551F661F771F2A95D2F7409560
:101D800050956095709503C040E050E0BA01C6954B
:101D9000C695C3708A019B01082B192B2A2B3B2B5C
:101DA000C901B801C23049F058F4C13019F00E949D
:101DB000A110CFC00E948F10CCC00E94B310C9C028
:101DC0000E948D10C6C0112319F08C2F817001C0A4
:101DD0008695882309F4BDC02D2F2295269527705E
:101DE000220F220F6D2F6F70862F90E0A0E0B0E0E1
:101DF000022E04C0880F991FAA1FBB1F0A94D2F796
:101E0000D4FF10C04FE050E060E070E004C0440F29
:101E1000551F661F771F2A95D2F7409550956095FC
:101E2000709503C040E050E0BA01C695C695C370F6
:101E30008A019B01082B192B2A2B3B2BC901B801C6
:101E4000C23049F058F4C13019F00E94661181C0C7
:101E50000E9454117EC00E9478117BC00E94C7105E
:101E600078C0CF70112339F08C2F0E94ED108D2F88
:101E70000E94920D6EC08D2F0E94990D8C2F0E9492
:101E80000E1167C0D23F21F128F4D03F41F0D13F7D
:101E9000C1F043C0D33F19F1D43F79F03EC01123C4
:101EA00041F0053008F051C08C2F8F710E94331122
:101EB0004CC0063008F049C0F7CF8091C50282FFC0
:101EC00018C0112339F08C2F8F710E94ED103DC086
:101ED0001123C9F38C2F8F710E940E1136C011236C
:101EE00029F08C2F8F710E94D8102FC00E94D31020
:101EF0002CC0112349F0CF718C2F0E94ED1063E0AC
:101F00008C2F0E940F1621C081E00E942A160230F9
:101F1000E0F082E00E942A1618C0112331F000235D
:101F200091F28D2F0E945B0C10C0002399F2D933DF
:101F300049F41FEF27EE33E0115020403040E1F725
:101F400000C000008D2F0E940A0D88EF8C0D843098
:101F500020F40E947D240E94C90BDD20C9F00E945C
:101F60007D1580FD15C0F70112820E9477150E9431
:101F7000ED10C7010E94E90F0E947715DF91CF9104
:101F80001F910F91FF90EF90DF90CF900C940E1166
:101F9000DF91CF911F910F91FF90EF90DF90CF9045
:101FA00008950F931F93CF93DF93EC01688179819C
:101FB0008A810E942F128C010E948A110E947B103C
:101FC000B801CE010E94A00DDF91CF911F910F911A
:101FD0000895CF93DF93EC01988189812B813C8117
:101FE000232B31F08F3F31F481E09F3F19F403C080
:101FF00081E001C080E080FD1DC0CE010E94230B66
:10200000811110C00E9481158823A1F08A81882344
:1020100089F08091C50282FD0DC082E0DF91CF91F1
:102020000C942A16CE010E94D10FCE01DF91CF91E0
:102030000C949E0ADF91CF91089580E090E00E9479
:10204000E02480E090E00E94F6240E94A8150E94FF
:10205000CA150E94F51E0C94421D809102019091B8
:1020600003010E9452250C941D100E9498150C9497
:102070002D1092959F70963079F010F4925001C017
:102080009A50923068F4803F69F018F4883E40F42A
:1020900009C0843F29F406C0883E20F0813F11F03A
:1020A00080E0089581E00895FC01808191810E9483
:1020B00024120E9439100895CF93DF9300D000D0EE
:1020C0001F92CDB7DEB70F900F900F900F900F902B
:1020D000DF91CF910895CF93DF9300D000D000D04F
:1020E000CDB7DEB726960FB6F894DEBF0FBECDBFD4
:1020F000DF91CF910895089508950C947C100C946D
:102100007D100E947F1060932F02709330028093A5
:102110003102909332020C941D100C9481100F9395
:102120001F9300912F0210913002209131023091C3
:102130003202602B712B822B932B1F910F910C94E9
:1021400081100F931F9300912F0210913002209164
:1021500031023091320260237123822393231F9135
:102160000F910C9481100F931F9300912F021091E7
:10217000300220913102309132026027712782278C
:1021800093271F910F910C9481100C947C100E9446
:10219000C51060932B0270932C0280932D029093B4
:1021A0002E020C941D1060E070E0CB010C94C7105F
:1021B0000F931F9341E050E060E070E08A019B01C3
:1021C00004C0000F111F221F331F8A95D2F7C901C7
:1021D000B8011F910F910C94C7100F931F9341E00A
:1021E00050E060E070E004C0440F551F661F771F89
:1021F0008A95D2F780912B0290912C02A0912D020A
:10220000B0912E028A019B01082B192B2A2B3B2B04
:10221000C901B8011F910F910C94C7100F931F9320
:1022200041E050E060E070E004C0440F551F661FBD
:10223000771F8A95D2F7409550956095709580915B
:102240002B0290912C02A0912D02B0912E028A01B6
:102250009B01082319232A233B23C901B8011F919D
:102260000F910C94C7100F931F9341E050E060E072
:1022700070E004C0440F551F661F771F8A95D2F780
:1022800080912B0290912C02A0912D02B0912E02F0
:102290008A019B01082719272A273B27C901B80172
:1022A0001F910F910C94C7100F931F9300912B0255
:1022B00010912C0220912D0230912E02602B712B57
:1022C000822B932B1F910F910C94C7100F931F9388
:1022D00000912B0210912C0220912D0230912E02A0
:1022E00060237123822393231F910F910C94C710B5
:1022F0000F931F9300912B0210912C0220912D021D
:1023000030912E0260277127822793271F910F910A
:102310000C94C71008952DE0929F800D1124E82F92
:10232000E695E695E695877051E001C0550F8A95D0
:10233000EAF785E0E89FF0011124E250FE4F20E02B
:1023400030E070E04081CB01022E02C09695879567
:102350000A94E2F7817081958427852384278193ED
:102360002F5F3F4F2530310569F708952DE0929F8B
:10237000800D1124682F669566956695982F977045
:1023800085E0689FB001112440E050E080E0FB014F
:10239000E40FF51FE250FE4F208130E0092E02C00D
:1023A000369527950A94E2F721703327042E01C051
:1023B000220F0A94EAF7822B4F5F5F4F4530510599
:1023C00031F70895BF92CF92DF92EF92FF920F9371
:1023D0001F93CF93DF938C01C0902B02D0902C02DF
:1023E000E0902D02F0902E0280912F029091300209
:1023F000A0913102B0913202C82AD92AEA2AFB2AD6
:10240000CFE1D0E0D701C6010C2E04C0B695A79548
:10241000979587950A94D2F780FD04C0219790F78D
:10242000B12C07C0BC2EB8018C2F0E943E19019719
:10243000A9F38B2DDF91CF911F910F91FF90EF901A
:10244000DF90CF90BF900895CF93DF93EC010E946F
:10245000E211BE010E943E19DF91CF9108951F93B2
:10246000CF93DF93EB019091FD01992321F0CB01F4
:102470000E94241213C0882349F0CB010E94E2116C
:10248000182F682FCE010E948B1104C0CB010E942F
:10249000B611182FBE01812F0E943E19DF91CF91F6
:1024A0001F9108951F93CF93DF93C091330216E0DD
:1024B00080913402C81799F0D0E01C9FF0011D9F55
:1024C000F00D1124EB5CFD4F4081518162817381DD
:1024D000848195810E946B102196C770E9CFDF91AE
:1024E000CF911F91089540916502509166026091CD
:1024F0006702709168028091690290916A020C945F
:102500006B10EF92FF920F931F93CF93DF93809105
:102510006A0282958F7009F065C0809167028823F6
:1025200009F460C080913302F0903402109165028A
:1025300000916602609168027091690291E01F3F0C
:1025400009F090E0C0910001D0910101292F96E09F
:10255000E92E8F1509F446C06115710521F00F3F72
:1025600021F030E003C031E001C0322F90E030FDB7
:1025700036C0E89EF001E99EF00D1124DF01AB5C4E
:10258000BD4F11963C911197301329C03C913113E6
:1025900026C012963C911297311121C013964D918D
:1025A0005C911497461B570B4C175D07C0F4809144
:1025B0006A028F70806180936A02E65CFD4F8081C1
:1025C0008F708061808385E692E00E94E90FDF9141
:1025D000CF911F910F91FF90EF900C9452120196A2
:1025E0008770B7CFDF91CF911F910F91FF90EF9040
:1025F00008959F92AF92BF92CF92DF92EF92FF9297
:102600000F931F93CF93DF93CDB7DEB761970FB6CC
:10261000F894DEBF0FBECDBF8C0185E0F801DE016E
:102620001D9601900D928A95E1F7D8011296EC90D3
:1026300090916502E09166022091680230916902F2
:102640002115310531F0EF3F31F481E09F3F19F45E
:1026500003C081E001C080E0B82FB1709B2E80FDE7
:1026600047C1D8014C9111965C9111971396AD908A
:10267000BC90149785E6C82E82E0D82EF0906702B1
:10268000B501621B730B2091000130910101FF2005
:1026900009F4D9C080916A026217730708F095C0E7
:1026A000282F207F09F052C05E1313C0491311C0B8
:1026B000FE2CE1100EC08F70806180936A020E9430
:1026C0007312C6010E94E90F80916A02F8018583A6
:1026D0004DC1AB2831F05F3F31F481E04F3F19F439
:1026E00003C081E001C080E080FD03C081E08E2551
:1026F00002C080E090E0F82FF170FF2E80FF1CC038
:10270000809133022091340236E0821709F40BC124
:1027100090E0389FF001399FF00D1124EB5CFD4FE4
:102720006181561306C06081461303C06281E612C0
:1027300003C001968770E9CFFE2CEE2009F416C184
:1027400080916A02816080936A0254C05E1306C061
:10275000491304C0E11002C0F80199C0C8010E94E9
:102760005410882361F1EE2051F120916A02822FEA
:1027700082958F7090E0029774F08091650290913D
:10278000660298878F831986BB86AA862C87CE011E
:1027900007960E94E90F86E0F801A5E6B2E00190F5
:1027A0000D928A95E1F70E9481120E9473120AC06D
:1027B0005E1711F1C8010E94541081112CC0C8018C
:1027C0000E94E90FFF24F394D1C0282F207F81F7C6
:1027D0007A2DB98AA88A6E2D89890E945C1085E6B7
:1027E00092E00E94E90F86E0D6011D928A95E9F7F2
:1027F0000E947312F12CBAC04913DCCFE110DACF7A
:10280000F8018583C8010E94E90F86E0D6011D9278
:102810008A95E9F7ABC0EE2091F220916A02822FEF
:1028200082958F7090E002970CF4B5CF809165028D
:10283000909166029A8389831B82BD82AC822E832B
:10284000CE010196A6CF6217730708F044C0FE2C94
:10285000EE2009F4B4CF5E1330C049132EC020918E
:102860006A0220FD21C0822F82958F70482F50E090
:1028700041155105C9F0F80125834F30510541F04C
:102880008F5F982F9295907F822F8F70892B8583F1
:10289000C8010E94E90F86E0F801A5E6B2E00190C8
:1028A0000D928A95E1F73CC086E0F801A5E6B2E01A
:1028B00001900D928A95E1F759C0C8010E94541009
:1028C000811169CF80916A02816080936A02C80198
:1028D0000E94E90F4BC07A2DB98AA88A6E2D89898A
:1028E0000E945C1086E0D6011D928A95E9F718C017
:1028F000EE2009F464CFC8010E945410F82E8823FA
:1029000009F45DCF86E0F801A5E6B2E001900D92F2
:102910008A95E1F785E692E00E94550C0E948112AB
:102920000E94731223C04D875E878D859E850E940D
:102930002412292F22952F70223028F49F7039F00D
:10294000811105C00BC0243028F49F7049F4805ECB
:10295000883020F0C8010E94E90F9F2CF92C06C096
:10296000D80115969C91907F91F7F8CF8F2D6196A5
:102970000FB6F894DEBF0FBECDBFDF91CF911F9190
:102980000F91FF90EF90DF90CF90BF90AF909F900E
:1029900008951F93CF93DF93CDB7DEB72C970FB673
:1029A000F894DEBF0FBECDBF4F83588769877A8703
:1029B0008B879C87CE0107960E94F9128823D1F05D
:1029C0009F8188852A853B85232B31F08F3F31F409
:1029D00081E09F3F19F403C081E001C080E080FDE9
:1029E00047C04F81588569857A858B859C850E9473
:1029F0006B103EC086E0FE013796DE011196019015
:102A00000D928A95E1F7FF81E8856A857B856115DE
:102A1000710531F0EF3F31F481E0FF3F19F403C05D
:102A200081E001C080E080FD23C02091340230E0CD
:102A3000C9010196877099274091330250E08417AD
:102A40009507F1F1F983EA837D836C8396E0929F89
:102A5000D001939FB00D1124AB5CBD4FFE013196A8
:102A600001900D929A95E1F7809334020E945212E0
:102A700016E08091330290913402891771F1189F0A
:102A8000C00111248B5C9D4F0E94F912882329F10B
:102A9000E09133021E9FF0011124EB5CFD4F408159
:102AA000518162817381848195810E946B10809134
:102AB000330290E001968770992780933302D9CF33
:102AC0000E9435101092340210923302E5E6F2E0D3
:102AD00086E0DF011D928A95E9F72C960FB6F894EF
:102AE000DEBF0FBECDBFDF91CF911F9108958091C2
:102AF00073028595859585950895809173028770F9
:102B0000089590917302977081E009F480E0089530
:102B100080917E02089590917E02892B80937E029F
:102B20000895809590917E02892380937E02089576
:102B300010927E02089590917D02892B80937D02F0
:102B40000895809590917D02892380937D02089558
:102B500010927D02089580917402089508950C9456
:102B6000AE150C94AF159091C50292FD08C09091DE
:102B70007402981721F0809374020C94B115089593
:102B800080917402882329F01092740280E00C94E2
:102B9000B1150895CF93DF93E0910201F091030105
:102BA00080917E028083E0910201F0910301908187
:102BB00080917D02892B808380917402882381F02B
:102BC000E0910201F09103019081892B8083809133
:102BD0000201909103010E940C2581110E94C015F1
:102BE000C0910201D091030148E050E06BE672E031
:102BF000CE010E94372E892B69F088E0FE01ABE6FA
:102C0000B2E001900D928A95E1F7CE01DF91CF916C
:102C10000C948924DF91CF9108950C94AE15909176
:102C2000C50292FD10C098E0899F90011124262BC7
:102C3000209373020E94ED10809173028595859513
:102C400085950C940D160C94ED101092730280E093
:102C50000C940D1620917302809582238093730249
:102C6000982F977099F430E0482F082E000C550BE0
:102C70002417350759F09091C50292FD07C085953C
:102C8000859585950E940E110C9425160895CF9375
:102C90009091C50292FB222720F92817F9F0C82F3E
:102CA000892FC0FB82F98093C5028091C402909164
:102CB000C5020E94A81682E00E942A168091910205
:102CC00080FF0CC01F92CF938FEA99E09F938F9360
:102CD0000E94F1090F900F900F900F90CF910895DF
:102CE0008091C50282FB882780F991E089270C94A6
:102CF000471681E00C94471680E00C94471680E05C
:102D000090E00E944C2E21E0893E9E4F09F020E089
:102D1000822F089582E090E00C94442E83E090E0AE
:102D20000C94442E682F83E090E00C94522ECF93A5
:102D300084E090E00E94442EC82F82E290E00E943E
:102D4000442E2C2F30E0A901582BCA01CF910895B1
:102D5000CF93C92F682F84E090E00E94522E6C2FF1
:102D600082E290E0CF910C94522EAB01BC018FE037
:102D700090E00C94642EAB01BC0183E190E00C94D4
:102D8000642E60E070E0CB010C94BB1660E070E054
:102D9000CB010E94B5160C94C11669EE7EEF80E05F
:102DA00090E00E94702E60E082E090E00E94522E3F
:102DB00060E083E090E00E94522E10922F02109269
:102DC0003002109231021092320260E084E090E012
:102DD0000E94522E60E082E290E00E94522E60E05B
:102DE00085E090E00E94522E60E086E090E00E9434
:102DF000522E6FEF87E090E00E94522E40E050E0AC
:102E0000BA0188E090E00E94642E60E08DE090E0DE
:102E10000E94522E40E050E0BA0188E190E00E940A
:102E2000642E60E087E190E00E94522E40E050E086
:102E3000BA018CE190E00E94642E60E070E080E2D4
:102E400090E00E94702E40E050E0BA0188E190E0EE
:102E50000E94642E0C94C6160C94CD16682F8EE03A
:102E600090E00C94522E0E94012660938D02709384
:102E70008E0280938F0290939002609389027093E8
:102E80008A0280938B0290938C02089585B78068A4
:102E900085BF85B7806885BF089581E008950C944B
:102EA0004D1708950C9451170C9451170C94541706
:102EB0000C9451170C9458170C9451170E944617F4
:102EC00087E498E20E9473240E945C170C945A17BE
:102ED0000E9452170C9451170E941B1A0C94C80B95
:102EE0000E94EC250E94441B0E946C170C945617FC
:102EF0005F926F927F928F929F92AF92BF92CF928A
:102F0000DF92EF92FF920F931F93CF93DF93CDB792
:102F1000DEB72A970FB6F894DEBF0FBECDBF0E9472
:102F2000591BC82E81110E9433173FE7832E32E0D0
:102F3000932E00E010E0502E802F0E943F1A5C017B
:102F4000F401619071904F01682679266114710433
:102F5000B1F40F5F1F4F0530110569F78FEF8983BB
:102F60008A831B820E94F5258160782F9D838C8344
:102F700049815A816B818D810E940B0C3AC08091EE
:102F8000910281FD0E94481AD12CEE24E394F12C89
:102F9000C3018E219F21892B29F10E944F1788237D
:102FA000A9F0DE825F82AE20BF2081E0AB2809F469
:102FB00080E088870E94F5258160782F9A8789872D
:102FC0004E815F8168858A850E940B0C000F111F5E
:102FD000F801E158FD4F80819181E826F926F182C0
:102FE000E08207C0D394EE0CFF1CFDE0DF12D0CFCF
:102FF000B0CF81E0C11001C080E02A960FB6F894EE
:10300000DEBF0FBECDBFDF91CF911F910F91FF901B
:10301000EF90DF90CF90BF90AF909F908F907F9078
:103020006F905F9008950E9478170E94E21D0C94A3
:10303000D90BCF93DF930E944319EC01811521E551
:10304000920708F045C0811530E5930708F094C059
:10305000883E910528F5803E910508F0F8C0883A31
:10306000910570F4853A910508F07CC08130910596
:1030700009F475C008F4E8C0049708F0E8C0E4C09B
:103080008F3B910508F0E0C0C85AD0E0CC0FDD1F9F
:10309000C65BDE4F0990D881C02DCE019464D8C0A4
:1030A000811540E2940758F4811551E0950708F026
:1030B000CEC08D3E910508F4C7C09065C9C0C1154A
:1030C00080E4D80708F4C0C0DF70CE01906AC0C0A9
:1030D000811525E59207A8F4811534E5930708F0DA
:1030E00095C0811543E5940708F07BC0811552E532
:1030F000950708F061C0D82FCC27CE01816F906A68
:10310000A7C0C11589E5D807A0F4C11528E5D207E5
:1031100008F082C0C11536E5D30708F095C08C2FA2
:103120000E94D7198F7190E0D82FCC27CE019062E2
:103130008FC0C1154AE5D40708F474C0CE0190567B
:103140008115904208F080C08D2F8F710E94D71991
:10315000DD27D0628F71AE01582BCA0179C081E0A2
:1031600090E076C0C55AD0E0C858DE4F8881C82F9D
:10317000D0E0CE0190646CC074E0969587957A9506
:10318000E1F7282F23703C2F337081E090E002C0DC
:10319000880F991F3A95E2F79C68AC01522B9A016F
:1031A0009C2F9F709695969550E2959FE001112473
:1031B000C9018C2B9D2B4CC08370992721E030E0F6
:1031C00002C0220F331F8A95E2F79C2F96959695A1
:1031D00080E2989FE0011124C22BD32BCE019C6882
:1031E00037C08370992721E030E002C0220F331FDF
:1031F0008A95E2F79C2F9695969540E2949FE00180
:103200001124C22BD32BCE019A6822C0D82FCC27F1
:10321000CE01846F906A1CC0DC2FCC27CE01806F5A
:10322000906A16C08C2F8F700E94D71994E0D695A3
:10323000C7959A95E1F7CF70D0E0DC2FCC27D06905
:103240009E01282BC90104C080E090E001C0CE019E
:10325000DF91CF91089521E4829FC0011124FC01E8
:103260002DE0729FE00DF11D1124E60FF11DEE0F10
:10327000FF1FE852FF4F8591949108950E942B19EA
:103280000E94191808958238910569F1B0F48133CC
:10329000910509F46DC048F48932910509F463C0C1
:1032A0008A32910509F469C008958533910509F4BE
:1032B00055C089339105B9F00895833E910569F1B0
:1032C00038F4803E9105B1F0823E910509F10895F0
:1032D000863E9105A9F1873E9105B9F1843E91059D
:1032E00009F064C023C02091C40220FD4FC021FD1D
:1032F0004DC008958091C40280FD44C08091C502F4
:1033000080FF44C08091C40284FD42C083EE4DC062
:103310008091C40282FF38C0F5CF8091C40282FD43
:1033200033C08091C50280FD31C0ECCF8091C502D1
:1033300081FF32C08091C40284FD2AC087EE35C06F
:103340008091C40283FF26C0F5CF8091C40283FD23
:1033500021C08091C50281FD1FC0ECCF8091C402C5
:1033600085FD1CC01DC08091C40285FD19C016C01A
:103370008091C40286FD16C017C08091C40286FDEC
:1033800013C010C089E311C082EE0FC080EE0DC0E3
:1033900080E00BC086EE09C084EE07C089E205C05C
:1033A00085E303C08AE201C081E390E00895909133
:1033B000C40292FF0DC0282F2871283019F4877F8E
:1033C000846006C0282F2471243011F48B7F88601C
:1033D00093FF0DC0282F2871283119F4877E84614E
:1033E00006C0282F2471243111F48B7E886120912E
:1033F000C50220FF0DC0382F3871383019F4877F8F
:10340000816006C0382F3171313011F48E7F8860B1
:1034100021FF0DC0282F2871283119F4877E816182
:1034200006C0282F2171213111F48E7E886194FD10
:10343000877E089508950E947F16811102C00E9420
:103440002C170E948A16809391020E9497169093DF
:10345000C5028093C4020E941A1A0E948E16682F19
:1034600070E080E090E00E948D1060912B027091DE
:103470002C0280912D0290912E020C94C510E82F01
:10348000F0E0EE0FFF1FE053FD4F80819181089522
:10349000CF92DF92EF92FF920F931F93CF93DF9320
:1034A00084ED99E00E94580980EDE82E82E0F82E24
:1034B000C0E0D0E09FECC92E99E0D92E06EC19E0CF
:1034C000DF93CF93DF92CF920E94F1098CEC99E0C9
:1034D0000E945809F701819191917F010E94AE0BE2
:1034E0009F938F931F930F930E94F10984EC99E0AF
:1034F0000E94580921968DB79EB708960FB6F8948A
:103500009EBF0FBE8DBFC530D105D1F6DF91CF91E3
:103510001F910F91FF90EF90DF90CF90089580EA78
:103520008A95F1F7089500C008950C948F1A0895B4
:103530000C94971A0C94981A0C94580AF894E82F43
:10354000E295EF70F0E031A1282F2F7081E090E03C
:1035500001C0880F2A95EAF7982F9095932391A39D
:1035600092A1892B82A3789408950F931F93CF93F0
:10357000DF93C8E8D1E089918F3F11F00E949E1A35
:1035800081E0CD38D807B9F7CBE7D1E008E811E002
:1035900089918F3F11F00E949E1A0C171D07C1F7E9
:1035A000DF91CF911F910F910895BF92CF92DF923B
:1035B000EF92FF920F931F93CF93DF938C01C62F4F
:1035C000D0E0CE0188579E4F6C01FC0190819F3F57
:1035D00009F450C0B62EF894E92FE295EF70F0E0B0
:1035E00081A19F7021E030E001C0220F9A95EAF797
:1035F000822B81A382A12095282322A378940E9464
:10360000931AEBE7F1E048E851E021E030E0E12CEB
:10361000F12C61916F3F89F0A62FA295AF70B0E0B9
:1036200090968C9190E06F7002C0959587956A9501
:10363000E2F780FD02C0C90102C080E090E0E82A04
:10364000F92A220F331F4E175F0719F7F601808101
:103650008F3F11F00E949E1A61E0E114F10409F419
:1036600060E08B2D0E94951ACC0FDD1FC00FD11F7B
:10367000F982E882DF91CF911F910F91FF90EF9037
:10368000DF90CF90BF9008950E94B51A8AE0E0EDD8
:10369000F2E0DF01982F1D929A95E9F7E6ECF2E04F
:1036A000DF011D928A95E9F785E00E94A41B0C9426
:1036B0000F0BFF920F931F93CF93DF93CDB7DEB71E
:1036C0002A970FB6F894DEBF0FBECDBF8E010F5FF5
:1036D0001F4F8AE0F80111928A95E9F7F12C6F2DBE
:1036E000C8010E94D51AF394F5E0FF12F8CF4AE022
:1036F00050E0B80186EC92E00E94372EFF24F3944C
:10370000009709F4F12C892B41F08AE0F801A6EC2E
:10371000B2E001900D928A95E1F72F2D45E060ED22
:1037200072E086EC92E00E94A51B0E94110B8F2D87
:103730002A960FB6F894DEBF0FBECDBFDF91CF91B2
:103740001F910F91FF9008950895FF920F931F937B
:10375000CF93DF93F82E092F162FD72FC42F2223B4
:1037600049F081E0809394020E94F52590939302A2
:1037700080939202809194028823D9F080919202E2
:10378000909193020E940D26059798F0EF2DF02F4F
:10379000A12FBD2F80E090E04C2F50E084179507BB
:1037A00034F4219131912D933D930196F7CF1092EE
:1037B0009402DF91CF911F910F91FF9008950E9485
:1037C000C3280E9470170C94CF280E94D3280E940F
:1037D00013180C94F1280E9493250E94AA280E9495
:1037E0005E170E94DF1B0E94E51B0E946817FBCF3B
:1037F00080919B0280FF06C06091090170E0660F16
:10380000771F26C081FF04C06091090184E005C0D4
:1038100082FF07C06091090188E0689FB001112410
:1038200017C090919A029923D1F0609108019617E0
:1038300088F72091090188E0289F90011124929F28
:10384000A001939F500D112470E0CA010E94092E1F
:103850006038710540F46115710519F406C068E01F
:1038600070E0862F08958FE7089581E00895809194
:103870009B0280FF08C06091050170E07595679517
:103880007595679521C081FF06C06091050170E0C4
:103890007595679519C082FF04C06091050170E0BD
:1038A00010C090919902992399F0609104019617A4
:1038B000A0F780910501899FC001112470E00E944A
:1038C000092E6038710540F46115710519F406C0C0
:1038D00061E070E0862F08958FE7089581E00895F4
:1038E0008D3E21F40E94F81B819504C08E3E29F480
:1038F0000E94F81B80939F0208958F3E21F40E943E
:10390000F81B819504C0803F29F40E94F81B809326
:103910009E020895893F19F40E94371C05C08A3F12
:1039200031F40E94371C81958093A00208958B3F4B
:1039300021F40E94371C819504C08C3F29F40E9419
:10394000371C8093A10208959FE0980F983078F477
:1039500021E030E0A90102C0440F551F9A95E2F71B
:10396000CA0190919D02892B80939D0208958D3FFD
:1039700021F480919B0281600BC08E3F21F48091E5
:103980009B02826005C08F3F29F480919B02846076
:1039900080939B0208958D3E39F490919F0297FF8A
:1039A00035C010929F0259C08E3E29F490919F021B
:1039B0001916BCF32BC090919E028F3E29F497FFFD
:1039C00025C010929E0249C0803F19F41916CCF30D
:1039D0001DC09091A002893F29F41916BCF41092E1
:1039E000A0023BC08A3F19F497FF10C0F8CF8B3F6D
:1039F00039F49091A10297FF09C01092A1022DC045
:103A00008C3F21F49091A1021916BCF39FE0980F0E
:103A1000983080F421E030E0A90102C0440F551F26
:103A20009A95E2F7CA01809590919D02892380932F
:103A30009D0213C08D3F21F480919B028E7F0BC0AD
:103A40008E3F21F480919B028D7F05C08F3F29F42A
:103A500080919B028B7F80939B0280919E028111BB
:103A600006C080919F02811102C010929A0280913B
:103A7000A002811106C08091A102811102C01092A2
:103A8000990208958091910283FF7EC082E19AE0BD
:103A90000E94580980919D021F928F938DE09AE0B9
:103AA0009F938F930E94F1098BE09AE00E9458093E
:103AB00080919E02282F082E000C330B3F938F938A
:103AC00088E09AE09F938F930E94F10986E09AE044
:103AD0000E94580980919F02282F082E000C330B5A
:103AE0003F938F9383E09AE09F938F930E94F10915
:103AF00081E09AE00E9458098091A002282F082EA8
:103B0000000C330B3F938F938EEF99E09F938F932D
:103B10000E94F1098CEF99E00E9458098091A1025E
:103B2000282F082E000C330B3F938F9389EF99E0D9
:103B30009F938F930E94F10986EF99E00E945809A4
:103B400080919A021F928F9383EF99E09F938F93B6
:103B50000E94F10981EF99E00E94580980919B022F
:103B60001F928F938EEE99E09F938F930E94F1099D
:103B70008BEE99E00E9458098DB79EB74C960FB610
:103B8000F8949EBF0FBE8DBF0E94F52520919E0226
:103B9000211104C020919F02222321F090939802CA
:103BA000809397022091A002211104C02091A102CC
:103BB000222321F090939602809395028CE992E063
:103BC0000C94D224EF92FF920F931F93CF93DF9325
:103BD00000D000D000D0CDB7DEB786E0ECE9F2E04F
:103BE000DE01119601900D928A95E1F7E0909E0218
:103BF000F0909F020091A0021091A10210929E02EB
:103C000010929F021092A0021092A102E11003C034
:103C1000FF2009F45DC080919702909198020E9464
:103C20000D26AC0190919A02992339F020910A0156
:103C300030E02417350758F04BC020910B018AE083
:103C4000289F900111242417350718F041C09F3F89
:103C500019F09F5F90939A02EE2061F00E94F81B8A
:103C60001E1414F09FEF01C091E0989F902D112435
:103C700090939E02FF2061F00E94F81B1F1414F025
:103C80009FEF01C091E0989F902D112490939F0287
:103C900030919E023323E1F020919F022223C1F054
:103CA00045EB3403C0011124992319F090939E022F
:103CB00003C081E080939E0235EB2303C0011124F1
:103CC000992319F090939F0203C081E080939F0293
:103CD000011103C0112309F45DC0809195029091F8
:103CE00096020E940D26AC0190919902992339F019
:103CF0002091060130E02417350758F04BC0209181
:103D000007018AE0289F900111242417350718F035
:103D100041C09F3F19F09F5F90939902002361F08B
:103D20000E94371C101614F09FEF01C091E0989F7D
:103D3000902D11249093A002112361F00E94371C52
:103D4000111614F09FEF01C091E0989F902D11245F
:103D50009093A1023091A0023323E1F02091A102BF
:103D60002223C1F045EB3403C0011124992319F03B
:103D70009093A00203C081E08093A00235EB23035F
:103D8000C0011124992319F09093A10203C081E08E
:103D90008093A10280919E0281110BC080919F02AD
:103DA000811107C08091A002811103C08091A102FE
:103DB00081110E94421DEB82FC820D831E8386E0EE
:103DC000FE013196ACE9B2E001900D928A95E1F7DF
:103DD00026960FB6F894DEBF0FBECDBFDF91CF9110
:103DE0001F910F91FF90EF900895ECE9F2E086E0CB
:103DF000DF011D928A95E9F710929A0210929902BA
:103E000010929B020895CF93DF93EC01FB01828116
:103E1000882309F43CC1C430FDE5DF0760F4CB3FE3
:103E20009CE5D90788F49E0122503C452431310598
:103E300008F02EC109C0C236EDE5DE0729F0C63A0A
:103E4000FDE5DF0709F024C10E9497169093C50293
:103E50008093C402C1318CE5D80709F4C6C008F0CC
:103E600042C0C930ECE5DE0709F49BC000F5C5305F
:103E70008CE5D80709F485C078F4C330ECE5DE079B
:103E800009F478C008F07AC0C230DC4509F0F5C00A
:103E90008091C4028160EFC0C7309CE5D90709F466
:103EA00078C008F07AC08091C4028061E4C0CD304F
:103EB000FCE5DF0709F487C058F4CB309CE5D9074F
:103EC00009F479C008F07BC08091C40288606FC09B
:103ED000CF30FCE5DF0709F480C008F082C0809194
:103EE000C402877FC8C0CE3F9CE5D90709F471C0E2
:103EF00000F5C531FCE5DF0709F485C068F4C3317E
:103F00009CE5D90709F475C008F095C00E943510EA
:103F10008091C4028F77AFC0CC3FFCE5DF07A9F1E9
:103F200008F054C0CB3FDC4509F0A7C08091C50222
:103F300040C0C230EDE5DE0709F489C058F4C11570
:103F40008DE5D80709F45AC008F069C08091C50210
:103F500082602FC0C236EDE5DE0709F47CC0C63AA8
:103F6000FDE5DF0709F481C0C330DD4509F085C0F8
:103F700080E06EC08091C40282607DC08091C402E6
:103F800016C08091C402886076C08091C5028260AC
:103F90004FC08091C40280626EC08091C402806470
:103FA0006AC00E9435108091C402806864C0846039
:103FB00062C081603DC08091C4028E7F5CC08091F0
:103FC000C4028D7F58C08091C40216C08091C50282
:103FD00018C08091C5028D7F2BC08091C4028F7E56
:103FE0004AC08091C4028F7D46C08091C4028F7BFD
:103FF00042C08091C402877F8B7F3DC08091C50203
:104000008D7F8E7F15C08091C40282FB222720F90C
:1040100091E0922790FB82F990FB83F92CC080916C
:10402000C502982F909591708E7F892B90FB81F916
:104030008093C50222C00E9435108091C40287FB84
:10404000222720F991E0922790FB87F914C081E0A4
:104050000E942E1712C08091C40284FB222720F9EF
:1040600091E0922790FB84F906C08091C402982FBA
:10407000909590FB80F98093C4028091C402909146
:10408000C5020E94A8160E94351080E001C081E0A0
:10409000DF91CF910895809104011F928F938091B9
:1040A00005011F928F93809108011F928F93809139
:1040B00009011F928F9380910A011F928F93809123
:1040C0000B011F928F9385E39AE09F938F930E9439
:1040D000F1098DB79EB70E960FB6F8949EBF0FBE2E
:1040E0008DBF0895883220F58E3108F068C08B307E
:1040F00091F1C0F4873009F0BEC081E080930B01DC
:1041000084E180930A018AE0809309018EE1809323
:10411000080188E08093050188E28093040187E923
:104120009BE0C6C0833109F443C0843169F1A3C068
:104130008F3409F49EC028F4893231F1883359F064
:104140009AC0813531F008F4D4C0823509F4A7C093
:1041500092C08FEFA5C089EB9BE00E9458090E9496
:104160004B201F9281E08F931F9288E08F9382EB08
:104170009AE09F938F930E94F1090F900F900F90F8
:104180000F900F900F9096C086EB9BE00E9458090D
:104190008091A602882309F4AAC01092A602109268
:1041A000A5021092A4021092A3021092A202B1C022
:1041B00088EA9BE00E9458090E944B207BC08D51E9
:1041C0008093A602833031F170F48130D1F08230D7
:1041D00009F03FC08AE091E09093A5028093A40289
:1041E0008AE991E01FC0853059F108F1863089F5E0
:1041F00084E091E09093A5028093A40285ED91E084
:1042000011C08BE091E09093A5028093A40281E914
:1042100091E008C089E091E09093A5028093A40208
:1042200086EA91E09093A3028093A20218C088E0EE
:1042300091E09093A5028093A40283EB91E0F2CFEA
:1042400085E091E09093A5028093A40282EC91E036
:10425000E9CF1092A60285EA9BE00E94580980915E
:10426000A602882309F455C01F928F9381EA9BE030
:104270000DC08AE015C084E99BE01AC097FF47C0D3
:10428000108280811F928F938EE89BE09F938F9383
:104290000E94F1090F900F900F900F900BC081E0DA
:1042A000E091A402F091A502309729F58BE89BE0FC
:1042B0000E9458092091A602222359F18091A2025E
:1042C0009091A302009711F48DE891E09F938F9352
:1042D0001F922F9382E89BE09F938F930E94F10996
:1042E0000F900F900F900F900F900F9016C080E0DE
:1042F000089586EFD5CF2081082E000C990B820FF0
:10430000911D8F3F910509F00CF4B8CF8FEF80839A
:10431000B8CF8EE79BE00E94580981E00895CF93C3
:10432000C82F1F928F938FEC9BE09F938F930E94D7
:10433000F10981E090E0A0E0B0E0BC01CD0104C053
:10434000660F771F881F991FCA95D2F70E948D109C
:104350000F900F900F900F90CF910C943510EF921B
:10436000FF920F931F93CF93DF938B3109F4EDC02E
:1043700008F08EC08B3009F4B1C008F078C08630E8
:1043800009F4AFC020F4853009F4BDC04EC18730B8
:1043900009F4C0C0883009F048C10E948E161F92EF
:1043A0008F9383EF9FE09F938F930E94F1090E9468
:1043B0008A1683FB992790F91F929F9382FB992776
:1043C00090F91F929F9381FB992790F91F929F93D9
:1043D000982F91701F929F931F928F938AEA9FE06C
:1043E0009F938F930E94F1090E94971687FB2227C3
:1043F00020F91F922F9386FB222720F91F922F93DB
:1044000085FB222720F91F922F9384FB222720F976
:104410001F922F9383FB222720F91F922F9382FB59
:10442000222720F91F922F9391FB222720F91F9218
:104430002F93292F21701F922F9381FB222720F980
:104440001F922F93282F21701F922F939F938F934A
:1044500085EC9EE09F938F930E94F1098DB79EB7E4
:1044600088960FB6F8949EBF0FBE8DBF35C08031C1
:1044700009F495C020F48E3009F47BC0D6C0863193
:1044800009F4A8C0893109F0D0C08FE39CE084C052
:104490008A32E1F060F4873209F4C3C028F48E3127
:1044A00008F4C3C08D51BEC0893269F1BEC08334E7
:1044B00048F48A3308F0B3C0853309F4B2C08833B6
:1044C00069F0B3C0833409F4ACC0AFC08EE990E1A9
:1044D0000E9458090E942C17C1E0ACC082E29DE006
:1044E0005BC080919102817F8E7F809391028BEFE0
:1044F0009CE00E9458098AE990E10E94580981E0F5
:104500008093A702E9CF8EE790E10E9458090E94AC
:10451000140BE2CF80919102C82FC095C170C0FBEF
:1045200080F980939102CC2329F082E790E10E94E8
:10453000580980C085E690E10E9458098091910257
:10454000897F877F80939102C7CF9091910291FBE1
:10455000CC27C0F981E0C827892FC0FB81F980935F
:104560009102CC2319F088E590E129C08AE490E11A
:1045700013C09091910292FBCC27C0F981E0C8272B
:10458000892FC0FB82F980939102CC2319F08BE331
:1045900090E115C08BE290E10E9458099DCF909167
:1045A000910293FBCC27C0F981E0C827892FC0FB7B
:1045B00083F980939102CC2351F08FE190E10E9426
:1045C00058098091910281608093910233C082E109
:1045D00090E1E2CF0E940126162F072FF82EE92E38
:1045E000D091C302C09118010E947D24EF92FF92E6
:1045F0000F931F931F92DF931F92CF931F928F935E
:1046000084ED9BE09F938F930E94F1098DB79EB735
:104610000C960FB6F8949EBF0FBE8DBF5DCF895329
:1046200001C080E00E948F2157CF80E190E10E947D
:104630005809C0E08C2FDF91CF911F910F91FF900F
:10464000EF90089580E008950C942223CF93C82F13
:104650008091A702813071F040F0823009F045C0AE
:104660008C2F0E94722081E046C00E948815823201
:10467000F1F504C00E948815823261F48C2F0E94EB
:104680002423811104C08C2F0E94AF212CC081E013
:1046900090E029C08C2F0E942223811123C0C431B5
:1046A000C9F058F4CB3069F0C031B9F482E080939E
:1046B000A70288E30E94722015C0C93259F0C8339E
:1046C00061F48BEF9CE00E9458098BEC9BE00E9408
:1046D000580908C01092A7020CC089EC9BE00E9408
:1046E000580907C081E0817006C01092A70280E0DF
:1046F00002C080E0F8CFCF910895CF93DF93863149
:104700009C4541F5EB010E948815982F8A812091E4
:10471000020130910301882379F09A7A81E009F44B
:1047200080E08093A802911102C069E201C065E3B4
:10473000C9010E944E250AC08091A802811102C0C1
:1047400069E201C065E3C9010E9450250E94CA15B3
:1047500080E001C081E0DF91CF9108950F931F9316
:10476000CF93DF93C42FD22FFC0182818823C9F01D
:104770004093AB020E94F5259093AA028093A90270
:1047800080E28C0F883008F057C0C77081E001C00C
:10479000880FCA95EAF7DF91CF911F910F910C9482
:1047A000920D8091AB02481330C08091A902909184
:1047B000AA020E940D26883C910538F510E21D0FD3
:1047C000CD17B9F080E28C0F883040F4C77081E0DB
:1047D00001C0880FCA95EAF70E94990D183028F594
:1047E00081E09D2F977001C0880F9A95EAF70E948B
:1047F000920D802F0E94890D1830F0F4D77081E05F
:1048000001C0880FDA95EAF70AC080E28C0F883081
:1048100098F4C77081E001C0880FCA95EAF7DF916C
:10482000CF911F910F910C94990D802FDF91CF9113
:104830001F910F910C94890DDF91CF911F910F91D2
:1048400008950F939C01CB01243F4CE5340731F1CF
:1048500088F4293DFCE53F07D9F02A3D4CE53407B3
:1048600079F1283D3C45A9F506E221EE41EE68EDDF
:104870007CE52BC0263FFCE53F07E1F0A8F0273F91
:104880003C4539F507E225EE46EE67EF7CE51DC0B5
:1048900007E225EE45EE69ED7CE517C006E221EE64
:1048A00040EE64EF7CE511C007E225EE44EE65EFD3
:1048B0007CE50BC006E221EE42EE66EF7CE505C02A
:1048C00008E221E045EE6AED7CE50E94AE2380E03F
:1048D00008C0FC018281882319F01092AB0201C04C
:1048E00081E00F9108959093FB018093FA01089560
:1048F0009093B1028093B0020895E091B002F091DC
:10490000B102309721F00190F081E02D099480E010
:104910000895EF92FF920F931F93CF93DF93E0914F
:10492000B002F091B1023097B1F18C010280F381B5
:10493000E02D09958091910282FF2DC080FF04C077
:1049400087EB90E10E945809E80118E081EBE82E1E
:1049500080E1F82E8091910280FF0BC088811F9228
:104960008F93FF92EF920E94F1090F900F900F909A
:104970000F90115021961111EDCF8091910280FF7F
:104980000AC08FEA90E1DF91CF911F910F91FF90C4
:10499000EF900C945809DF91CF911F910F91FF90E8
:1049A000EF900895E091B002F091B102309739F0A4
:1049B00022E0DC012C930480F581E02D0994089518
:1049C0002091AE023091AF022817390771F0909311
:1049D000AF028093AE02E091B002F091B102309745
:1049E00021F00680F781E02D099408952091AC0212
:1049F0003091AD022817390771F09093AD02809382
:104A0000AC02E091B002F091B102309721F0008445
:104A1000F185E02D09940895FC01329697E080E03D
:104A2000915029F021912223D9F38F5FF9CF089576
:104A3000662349F0FC01329608962191621729F00D
:104A4000E817F907D1F780E0089581E008959C0107
:104A5000FC0132969FEF80E04191461789F09F3F1D
:104A600019F4411101C0982F8F5F8630A9F79F3F3D
:104A700039F0F901E90FF11D97FDFA956283089568
:104A800008959C012A5F3F4FFC014281461301C0FB
:104A90001282019682179307B9F708950C9427257F
:104AA0000C944125029626E0FC0111922A95E9F723
:104AB000089508950C94592583E08093B2020C94D4
:104AC0005A25811102C081E001C082E08093B202C8
:104AD0000C945A250C94612581E08093B2020C94C9
:104AE0005A250C946C2508950C9473250C94742508
:104AF0000C9473250C9473250C947325CF930E940A
:104B00007A250E94591B0E947825C0E08C2F0E94B4
:104B10003F1A892B29F4CF5FC530C1F780E001C06F
:104B200081E0CF91089508951F920F920FB60F92D2
:104B300011248F939F93AF93BF938091B302811100
:104B400013C08091DA029091DB02A091DC02B09157
:104B5000DD024196A11DB11D8093DA029093DB0224
:104B6000A093DC02B093DD02BF91AF919F918F9132
:104B70000F900FBE0F901F9018958091E202843025
:104B800031F10E94940B1092B30220E488E190E08E
:104B90000FB6F894A895809360000FBE2093600034
:104BA00083B7817F846083BF83B7816083BF78943C
:104BB000889583B78E7F83BF0FB6F894A8958091B0
:104BC0006000886180936000109260000FBE0895BD
:104BD0000E9435100C94980B82E084BD93E095BD43
:104BE0009AEF97BD80936E0008952FB7F894809147
:104BF000DA029091DB02A091DC02B091DD022FBFBE
:104C000008952FB7F8946091DA027091DB028091D9
:104C1000DC029091DD022FBF08959C014FB7F894FC
:104C20008091DA029091DB02A091DC02B091DD026A
:104C30004FBF821B930B089578941F920F920FB66B
:104C40000F9211248F939F93AF93BF938091DA02B9
:104C50009091DB02A091DC02B091DD020196A11DD2
:104C6000B11D8093DA029093DB02A093DC02B09333
:104C7000DD02BF91AF919F918F910F900FBE0F906A
:104C80001F901895F89481E08093E00080E2809373
:104C9000D800E9ECF0E010828FE19EE40197F1F793
:104CA00000C000001DBA109268001CBC10BE1FBAE4
:104CB00010927A0010926E0010926F0010927100A4
:104CC000109272001082ECEBF0E0108214B817B86A
:104CD0001AB81DB810BA108215B818B81BB81EB88B
:104CE00011BA0C94003F08958091C202089508956E
:104CF00022E02093E9002FEF3091E800215035FDAC
:104D000006C035ED3A95F1F700002111F5CF20915D
:104D1000E80025FF0BC040E050E066E070E00E9434
:104D200060298091E8008E778093E8000895CF9302
:104D3000DF9321E02093E9002FEF3091E80021502C
:104D400035FD06C035ED3A95F1F700002111F5CF9C
:104D50002091E80025FF14C0EC0140E050E068E03D
:104D600070E00E9460298091E8008E778093E800CF
:104D700088E0FE01AAEBB2E001900D928A95E1F77E
:104D8000DF91CF9108958093B6027093B80260933B
:104D9000B7028091E202843001F582E08093E9005D
:104DA0008FEF9091E800815095FD06C095ED9A95A2
:104DB000F1F700008111F5CF8091E80085FF0DC06B
:104DC00040E050E063E070E086EB92E00E946029F2
:104DD0008091E8008E778093E8000895BC0184E01C
:104DE0000C94C326BC0183E00C94C3268DED90E1A6
:104DF0000E9458098091E102811109C00E94F12AA4
:104E00000E944E2B8091E20084608093E20008951E
:104E100089ED90E10E9458091092E102089585ED14
:104E200090E10E9458090C94712581ED90E10E9457
:104E300058096091DE0281E0611101C080E00C94AC
:104E40005C258DEC90E10E9458099091E20281E08E
:104E5000943009F080E06091DE020C94612520918D
:104E6000B5022F5F822F62E30E94FD2D992319F076
:104E70002093B50208951092B5028091B90288235B
:104E800071F18091E202843041F58091E9008F70E8
:104E90002091EC00922F917020FD90E8892B93E0F7
:104EA0009093E9009091EB0090FF14C09091EE0078
:104EB00097FF10C09091E80095FF03C01092F10099
:104EC000F9CF9091E80090FF05C09091E8009E779F
:104ED0009093E8008F708093E9001092B9020895D2
:104EE00042E061EC81E00E946A2A42E261EC82E0E9
:104EF0000E946A2A42E261EC83E00E946A2A909151
:104F0000E20281E0943009F080E06091DE020C94CE
:104F10006A258091E402833009F461C030F4813065
:104F200071F0823009F49AC008958A3009F486C07D
:104F30008B3009F46CC0893009F0A8C020C0809182
:104F4000E302813A09F0A2C08091E800877F809354
:104F5000E8008091E7029091E802892B21F468E053
:104F60008AEB92E003C060E080E090E070E00E9495
:104F7000AB298091E8008B778093E80008958091B9
:104F8000E302813209F082C08091E7029091E80249
:104F9000029708F07BC08091E800877F8093E8004B
:104FA0008091E80082FD05C08091E2028111F8CF76
:104FB0006DC02091F3008091F20090E0922B029757
:104FC00031F48091F100813011F0863021F480912C
:104FD000F1008093C2028091E8008B7753C08091EA
:104FE000E302813A09F052C08091E7029091E80211
:104FF000892B09F04BC08091E800877F8093E800FF
:105000008091E80080FFFCCF8091180136C080912C
:10501000E3028132D9F58091E7029091E802892B71
:10502000A9F58091E800877F8093E8000E949F2A7D
:105030008091E502809318010C9435108091E30271
:10504000813221F58091E800877F8093E8000E94FB
:105050009F2A8091E6028093C30208958091E30223
:10506000813AA1F48091E800877F8093E8008091E5
:10507000E80080FFFCCF8091C3028093F100809113
:10508000E8008E778093E8000C949F2A08959FB7DC
:10509000F8941092B9029FBF9091E202943009F007
:1050A00057C09091E9009F703091EC00232F217040
:1050B00030FD20E8922B23E02093E9002091EB00C3
:1050C00020FF43C02091EE0027FF3FC02091B40293
:1050D000222321F02091E80025FF37C01092B4026E
:1050E00026E03091E80035FD15C03091E202343001
:1050F00061F53091EB0035FD28C0215021F481E0AD
:105100008093B40222C0EFE9FFE03197F1F700C0CD
:105110000000E7CF8093F1008091E80085FD0AC090
:105120008091E80080FFFCCF8091E8008E7780932B
:10513000E80006C08FB7F89421E02093B9028FBF32
:105140009F709093E90080E008959F709093E9002C
:105150008FEF089584B7877F84BF0FB6F894A89522
:1051600080916000886180936000109260000FBEA3
:1051700090E080E80FB6F89480936100909361000E
:105180000FBE0C946C250E94F12A0E944E2BE2EE79
:10519000F0E080818460808378940C94E22D8CE030
:1051A00091E00C9478248091E2028530C9F489EC76
:1051B00090E10E9458098091E202853079F40E94C2
:1051C000BD258091E0028823B1F30E947E258823CB
:1051D00091F30E944A290E943510EDCF0C94E825E6
:1051E000089508950C94F428292F3327233031058E
:1051F000C9F060F42130310581F02230310509F029
:1052000041C08BE590E02FE031E140C02132310513
:10521000E1F02232310531F135C082E190E02AE639
:1052200031E134C099278130910549F028F0029787
:1052300049F5E1EEF0E105C0EBE0F1E102C0E9EF94
:10524000F0E1849190E09F0121C063307105D0F4BA
:10525000660F771FFB01ED50FE4F2081318189E001
:1052600090E014C06330710568F4FB01EE0FFF1F7E
:10527000E351FE4F20813181FB01E651FE4F8081D9
:1052800090E004C080E090E020E030E0FA0131835B
:105290002083089580E189BD82E189BD09B400FEC3
:1052A000FDCF8091D8008F7D8093D8008091E00061
:1052B00082608093E0008091E00081FDFCCF089542
:1052C000CF92DF92EF92FF920F931F93CF93DF93D2
:1052D000EC018B017A010E94BE2A811133C0E114D6
:1052E000F10439F0F70180819181081B190BC80F77
:1052F000D91FC12CD12C0115110519F18091E8009D
:1053000085FD16C08091E8008E778093E800E11457
:10531000F10449F0F70180819181C80ED91ED18234
:10532000C08285E00FC00E94BE2A882321F30AC0F4
:1053300089918093F10001501109FFEFCF1ADF0A24
:10534000DACF80E0DF91CF911F910F91FF90EF9026
:10535000DF90CF9008952091E9023091EA0226175C
:10536000370748F06115710539F42091E8002E7770
:105370002093E80001C0B901FC0120E0611571052E
:1053800079F18091E2028823F1F18530F1F1809189
:10539000E80083FD3CC08091E80082FD2EC0809132
:1053A000E80080FFEBCF2091F3008091F20090E0C5
:1053B000922B6115710551F08830910538F42191D7
:1053C0002093F100615071090196F3CF21E0089715
:1053D00009F020E08091E8008E778093E800CECF3E
:1053E0002111CFCF0AC08091E202882361F085307D
:1053F00061F08091E80083FD0AC08091E80082FF9F
:10540000F2CF80E0089582E0089583E0089581E07E
:1054100008952091E9023091EA022617370748F0F3
:105420006115710539F42091E8002E772093E8008A
:1054300001C0B901FC0120E06115710591F1809175
:10544000E202882309F440C0853009F43FC080910E
:10545000E80083FD3DC08091E80082FD2FC080916F
:10546000E80080FFE9CF2091F3008091F20090E006
:10547000922B6115710559F08830910540F4249103
:105480002093F1003196615071090196F2CF21E02D
:10549000089709F020E08091E8008E778093E8007B
:1054A000CBCF2111CCCF0AC08091E202882361F0DA
:1054B000853061F08091E80083FD0AC08091E800AA
:1054C00082FFF2CF80E0089582E0089583E008959E
:1054D00081E00895982F973068F59093E900981728
:1054E00039F07091EC002091ED005091F00003C074
:1054F000242F762F50E021FD02C09F5FECCF30912A
:10550000EB003E7F3093EB003091ED003D7F309318
:10551000ED003091EB0031603093EB007093EC00C4
:105520002093ED005093F0002091EE0027FDE5CF91
:1055300080E008958F708093E90081E00895809164
:10554000E30287FF11C08091E80082FD05C08091D1
:10555000E2028111F8CF11C08091E8008B770BC077
:105560008091E202882349F08091E80080FFF8CF23
:105570008091E8008E778093E80008952091E40000
:105580003091E50095E64091EC00842F817040FF5A
:1055900023C08091E80080FD1DC08091E202882335
:1055A00099F0853099F08091EB0085FD11C0409114
:1055B000E4005091E5002417350729F3915011F0CC
:1055C0009A01E1CF84E0089582E0089583E0089590
:1055D00081E0089580E008954091E80042FFDDCF2A
:1055E00008950E945F2B0E94672BE0EEF0E080811F
:1055F00081608083E8EDF0E080818F77808319BC43
:10560000A7EDB0E08C918E7F8C9380818F7E80831C
:105610001092E10208950F931F93CF93DF930E949E
:105620005F2B0E94672BC8EDD0E088818F7788833D
:1056300088818068888388818F7D888319BC1092D7
:10564000E2021092DE021092E0021092DF0200EEFF
:1056500010E0F80180818B7F80838881816088835E
:1056600042E060E080E00E946A2AE1EEF0E08081A2
:105670008E7F8083E2EEF0E0808181608083808194
:1056800088608083F80180818E7F8083888180613B
:105690008883DF91CF911F910F910895E8EDF0E09D
:1056A00080818F7E8083E7EDF0E080818160808360
:1056B00084E082BF81E08093E1020C940B2BE8ED43
:1056C000F0E080818E7F80831092E2000895109236
:1056D000DA001092E10008951F920F920FB60F9218
:1056E00011242F933F934F935F936F937F938F93E7
:1056F0009F93AF93BF93EF93FF938091E10082FF5D
:105700000BC08091E20082FF07C08091E1008B7F97
:105710008093E1000E942F278091DA0080FF1FC054
:105720008091D80080FF1BC08091DA008E7F80932B
:10573000DA008091D90080FF0DC080E189BD82E14F
:1057400089BD09B400FEFDCF81E08093E2020E9492
:10575000F62605C019BC1092E2020E94082780912B
:10576000E10080FF19C08091E20080FF15C08091A8
:10577000E2008E7F8093E2008091E200806180935E
:10578000E2008091D80080628093D80019BC85E047
:105790008093E2020E9415278091E10084FF30C0CF
:1057A0008091E20084FF2CC080E189BD82E189BD47
:1057B00009B400FEFDCF8091D8008F7D8093D80082
:1057C0008091E1008F7E8093E1008091E2008F7EE6
:1057D0008093E2008091E20081608093E2008091FA
:1057E000DE02882311F084E007C08091E30087FD8A
:1057F00002C081E001C083E08093E2020E94212781
:105800008091E10083FF29C08091E20083FF25C0E1
:105810008091E100877F8093E10082E08093E20243
:105820001092DE028091E1008E7F8093E1008091F2
:10583000E2008E7F8093E2008091E200806180939D
:10584000E20042E060E080E00E946A2A8091F0007D
:1058500088608093F0000E940F27FF91EF91BF9125
:10586000AF919F918F917F916F915F914F913F91F8
:105870002F910F900FBE0F901F9018951F920F92AF
:105880000FB60F9211242F933F934F935F936F9313
:105890007F938F939F93AF93BF93CF93DF93EF93B8
:1058A000FF93C091E900CF708091EC00D82FD170A8
:1058B00080FDD0E81092E9008091F000877F80930E
:1058C000F00078940E94822C1092E9008091F00000
:1058D00088608093F000CD2BCF70C093E900FF91DA
:1058E000EF91DF91CF91BF91AF919F918F917F9178
:1058F0006F915F914F913F912F910F900FBE0F903D
:105900001F9018951F93CF93DF93CDB7DEB7AA975B
:105910000FB6F894DEBF0FBECDBFE3EEF2E080918C
:10592000F100819322E0EB3EF207C9F70E9489273C
:105930008091E80083FF2EC18091E3029091E40200
:10594000492F50E04A30510508F024C1FA01EE59C0
:10595000FF4F0C941D2E803821F0823809F01AC1B7
:1059600008C08091DF029091E002992389F0826063
:105970000FC08091E7028F70873008F00BC18093D1
:10598000E9008091EB0085FB882780F91092E900FF
:105990009091E800977F9093E8008093F100109237
:1059A000F100D1C0282F2D7F09F0F4C0882319F011
:1059B000823061F0EFC08091E502813009F0EAC0E9
:1059C000933009F080E08093E0022EC08091E502E0
:1059D00081112AC08091E7028F702FEF280F2630A7
:1059E00008F0D8C08093E9002091EB0020FF1CC094
:1059F000933021F48091EB00806214C09091EB0011
:105A000090619093EB0021E030E0A90102C0440FC7
:105A1000551F8A95E2F74093EA001092EA008091C0
:105A2000EB0088608093EB001092E9008091E80021
:105A3000877F8093E8000E949F2AACC08111AAC092
:105A40001091E5021F778091E3008078812B80938D
:105A5000E3008091E800877F8093E8000E949F2AFE
:105A60008091E80080FFFCCF8091E3008068809304
:105A7000E300111102C082E001C083E08093E202E2
:105A800089C08058823008F085C08091E5029091ED
:105A9000E6028C3D53E0950779F583E08A838AE23C
:105AA00089834FB7F894DE01139620E03EE051E27F
:105AB000E32FF0E050935700E49120FF03C0E295FC
:105AC000EF703F5FEF708E2F90E0EA3010F0C796D6
:105AD00001C0C0968D939D932F5F243149F74FBF2E
:105AE0008091E800877F8093E8006AE270E0CE0151
:105AF00001960E94AB2916C06091E7027091E802FE
:105B0000AE014F5F5F4F0E94F228BC01892B09F460
:105B100041C09091E800977F9093E80089819A8135
:105B20000E94092A8091E8008B778093E80032C0B8
:105B3000803881F58091E800877F8093E80080912C
:105B4000DE028093F1008091E8008E7772CF8111A0
:105B500021C08091E5029091E60299270297D4F442
:105B60008091E800877F8093E8008091E502809330
:105B7000DE020E949F2A8091DE02811106C0809180
:105B8000E30087FD02C081E001C084E08093E2026F
:105B90000E9470278091E80083FF0AC08091E8008E
:105BA000877F8093E8008091EB0080628093EB0018
:105BB000AA960FB6F894DEBF0FBECDBFDF91CF918E
:105BC0001F910895CF938091E2028823A1F0C091A4
:105BD000E900CF709091EC00892F817090FD80E8F2
:105BE000C82B1092E9008091E80083FD0E94822C6E
:105BF000CF70C093E900CF910895991B79E004C05C
:105C0000991F961708F0961B881F7A95C9F78095FB
:105C1000089597FB072E16F4009407D077FD09D05E
:105C20000E94232E07FC05D03EF4909581959F4F4E
:105C30000895709561957F4F0895EE0FFF1F0590B1
:105C4000F491E02D0994AA1BBB1B51E107C0AA1FC8
:105C5000BB1FA617B70710F0A61BB70B881F991F0D
:105C60005A95A9F780959095BC01CD010895FB0147
:105C7000DC0104C08D910190801921F44150504005
:105C8000C8F7881B990B0895F999FECF92BD81BD85
:105C9000F89A992780B50895A8E1B0E042E050E075
:105CA0000C94782E262FF999FECF92BD81BDF89ADB
:105CB000019700B4021639F01FBA20BD0FB6F89450
:105CC000FA9AF99A0FBE08950396272F0E94532E31
:105CD0000E94522E252F0E94532E242F0C94532EB7
:105CE0000196272F0E94532E0C94522EDC01CB01DB
:105CF000FC01F999FECF06C0F2BDE1BDF89A3196DC
:105D000000B40D9241505040B8F70895F894FFCF79
:105D1000C8007502280850011E0A1401742697262F
:105D20007826F226EE26772601E200E900EA00B5A1
:105D300000B600B700CD008301CC008A0192019427
:105D4000012102230224022502260227022A02B38D
:105D500000B4006F007000818283E200E900EA0075
:105D6000B500B600B700CD008301CC008A019201D6
:105D700094012102230224022502260227022A027C
:105D8000B300B4006F0070008182836697C634351B
:105D900036323331F7F6F5F493929190943F3F3FCA
:105DA000006D6B5F64656C6179006D6B5F696E742B
:105DB000657276616C006D6B5F6D61785F737065A5
:105DC0006564006D6B5F74696D655F746F5F6D61B5
:105DD00078006D6B5F776865656C5F6D61785F7388
:105DE00070656564006D6B5F776865656C5F74698D
:105DF0006D655F746F5F6D617800407B2219129E44
:0A5E0000117C1121113A1153110019
:00000001FF
